:1000000000308A000428000084011F308305831615
:100010001F129F121B0880399B0007309C001F1283
:100020009F121B0880399B0083121F1094128316A5
:100030000611861406120030831294008316940071
:100040000108C73908388100831290010030F80098
:10005000920000308316920007309C001C08831227
:100060000D1383169D018F010F08061083120614CD
:100070009930F700F70B3A2800000000831686102D
:10008000831286149930F700F70B44280000000013
:100090008316061183120615A1012108643C031C76
:1000A000672883160511831205150230F700F70B38
:1000B0005728000000008316051183120511023035
:1000C000F700F70B612800000000A10A4D288316F5
:1000D0000610831206109930F700F70B6D28000008
:1000E000000083168610831286109930F700F70BF4
:1000F000772800000000831606118312061199303C
:10010000F700F70B812800000000831635286300F4
:04400E00193FFC3F1B
:00000001FF
